:020000040000FA
:0A0000000000000066EF00F07ED063
:08001800CBD00F6A0E6EFF0E43
:100020000E260F2200D0D8A01200030E0B6EE60E93
:1000300002D8F5D70B6AFE0F0A6EE86A0B5AD8A0F1
:10004000120000000A0600D0F8D70DC01AF00CC04C
:1000500019F00BC018F00AC017F019501002F3CFB6
:100060000CF0F4CF0DF018501102F3500C26F450A0
:100070000D2217501202F3500C26F4500D221A5084
:100080001002F3500D2619501102F3500D2618508E
:100090001202F3500D2617501302F3500D2617507D
:1000A0001002F3CF0AF0F4CF0BF018501002F35007
:1000B0000B26F4500C22000E0D2217501102F350A3
:1000C0000B26F4500C22000E0D221200006A4F0E77
:1000D000AF6E240EAC6E900EAB6E00010F0EC16EB3
:1000E000070EB46E0FEE7FF0ED6AE950EA10FCE106
:1000F000EF6AC69AC30E926EE00E936EC00E946EB7
:10010000928092826ED0F2A403D0F294817A110090
:100110009EAA19D0060EAB1412E1E2CF4AF0E1CF4D
:1001200049F04B2A10EE6DF04B50E126000EE22212
:10013000AECFE7FF4AC0E2FF49C0E1FF1100AE5079
:10014000AE50AB98AB8811004B504C5C14E04C2A7D
:10015000EACF0BF0E9CF0AF000EE6DF04C50E92643
:10016000000EEA22EF500A6E0BC0EAFF0AC0E9FF58
:10017000D880120004D0E8680A6ED8A012001200DD
:100180004B6A4C6A9D8A9F8AF28EF28C12009D9A6D
:1001900000EE6DF0010EF46EF36AF306000EF45AF1
:1001A000EE6AF450F310F9E14B6A4C6A9D8A120032
:1001B000F29EE0CF6DF8D8CF6EF8E8CF6FF8F28EF0
:1001C0000001A192B36AB26AF29E6DC8E0FF6EC8E8
:1001D000D8FF6FC8E8FFF28E10009EA8FED7AD6E64
:1001E000120092988998939A8A8A0A0E16DF939A37
:1001F0008A9A9298899893948A9494948B949496DA
:100200008B96949A8B9A94988B98929A899A9490B8
:100210008B9094928B922C6A2A6A00EE4DF0200EFD
:10022000EE68E82EFDD72B6AABDFB1DFCD6AF29422
:10023000F28A870ED56EB16AA192A082B36AB26AC1
:10024000D08EA292B10EB16E06EC07F007EC0BF067
:1002500006EC0DF0B20EC1DF420EBFDF000EBDDFB7
:10026000422AE86A42B2010F43B0010806E1437036
:100270003E2A000E3F224022412266DF1B6EC30E43
:100280001B5C07E3FE0E1B5C01E301D01D6A56EF09
:1002900004F01BAE38D01D6A820E1B5C05E11BC04A
:1002A0001DF01E681F682DD0920E1B5C05E11BC05F
:1002B0001DF02068216825D0A20E1B5C05E11BC043
:1002C0001DF0226823681DD0B20E1B5C05E11BC027
:1002D0001DF02468256815D0C20E1B5C04E11BC00C
:1002E0001DF026680ED0D20E1B5C04E11BC01DF071
:1002F000276807D0E20E1B5C04E11BC01DF02868D4
:10030000296855EF04F01D5204E156EF04F055EF53
:1003100004F0820E1D5CD8A477D01E2803E11BC018
:100320001EF06ED01BC01FF0240E1E5C0AE3650E8B
:100330001E5C07E2820E51DF1E504FDF1F504DDF63
:100340005CD0780E1E5C0AE37C0E1E5C07E2820E17
:1003500044DF1E5042DF000E40DF4FD07C0E1E5C9B
:1003600008E18B9A2A922C9254685368526851681B
:1003700044D07D0E1E5C08E1899A2A942C9458681A
:1003800057685668556839D07E0E1E5C08E18B9020
:100390002A962C965C685B685A6859682ED07F0E46
:1003A0001E5C08E18B922A982C9860685F685E68F2
:1003B0005D6823D0750E1E5C08E18B942A9A2C9AF6
:1003C000646863686268616818D0760E1E5C08E134
:1003D0008B962A9C2C9C68686768666865680DD057
:1003E000770E1E5C08E18B982A9E2C9E6C686B68C9
:1003F0006A68696802D056EF04F01E6855EF04F091
:1004000056EF04F055EF04F0920E1D5CD8A4F4D121
:10041000202803E11BC020F0EDD11BC021F02152A8
:10042000D8A46AD0240E205C0AE3650E205C07E2A3
:10043000920ED3DE2050D1DE000ECFDE5BD0780EE0
:10044000205C0AE37C0E205C07E2820EC6DE2050B0
:10045000C4DE000EC2DE4ED07C0E205C08E18B9A1A
:100460002A922C92546853685268516843D07D0E8A
:10047000205C08E1899A2A942C9458685768566839
:10048000556838D07E0E205C08E18B902A962C9619
:100490005C685B685A6859682DD07F0E205C08E163
:1004A0008B922A982C9860685F685E685D6822D09D
:1004B000750E205C08E18B942A9A2C9A6468636814
:1004C0006268616817D0760E205C08E18B962A9CE2
:1004D0002C9C68686768666865680CD0770E205C3D
:1004E00008E18B982A9E2C9E6C686B686A68696824
:1004F00001D0DCD1DAD17ED12BA07AD1240E205CC0
:100500000AE3650E205C07E2920E67DE205065DE8E
:10051000215063DE6DD1780E205C0AE37C0E205CF6
:1005200007E2920E5ADE205058DE7F0E56DE60D172
:100530007C0E205C2FE121C02FF08B8A7F0E2F5C78
:1005400022E22C8202EE6DF0D8902F34E926000EC4
:10055000EA22EECF06F0EFCF07F006503E24026EFF
:1005600007503F20036E000E4020046E000E412015
:10057000056E05C054F004C053F003C052F002C031
:1005800051F02A8206D02C922A92546853685268FD
:1005900051682ED17D0E205C2FE121C030F0898A78
:1005A0007F0E2F5C22E22C8402EE6DF0D890303466
:1005B000E926000EEA22EECF06F0EFCF07F0065054
:1005C0003E24026E07503F20036E000E4020046E52
:1005D000000E4120056E05C058F004C057F003C05E
:1005E00056F002C055F02A8406D02C942A945868FC
:1005F000576856685568FCD07E0E205C2FE121C0FC
:1006000031F08B807F0E315C22E22C8602EE6DF0A1
:10061000D8903134E926000EEA22EECF06F0EFCF73
:1006200007F006503E24026E07503F20036E000E76
:100630004020046E000E4120056E05C05CF004C031
:100640005BF003C05AF002C059F02A8606D02C96FF
:100650002A965C685B685A685968CAD07F0E205C2D
:100660002FE121C032F08B827F0E325C22E22C8897
:1006700002EE6DF0D8903234E926000EEA22EECF79
:1006800006F0EFCF07F006503E24026E07503F20E1
:10069000036E000E4020046E000E4120056E05C062
:1006A00060F004C05FF003C05EF002C05DF02A8815
:1006B00006D02C982A9860685F685E685D6898D05C
:1006C000750E205C2FE121C033F08B847F0E335CEC
:1006D00022E22C8A02EE6DF0D8903334E926000E27
:1006E000EA22EECF06F0EFCF07F006503E24026E6E
:1006F00007503F20036E000E4020046E000E412084
:10070000056E05C064F004C063F003C062F002C06F
:1007100061F02A8A06D02C9A2A9A64686368626813
:10072000616866D0760E205C2FE121C034F08B86A4
:100730007F0E345C22E22C8C02EE6DF0D8903434C3
:10074000E926000EEA22EECF06F0EFCF07F00650C2
:100750003E24026E07503F20036E000E4020046EC0
:10076000000E4120056E05C068F004C067F003C0AC
:1007700066F002C065F02A8C06D02C9C2A9C686822
:1007800067686668656834D0770E205C2FE121C009
:1007900035F08B887F0E355C22E22C8E02EE6DF0F8
:1007A000D8903534E926000EEA22EECF06F0EFCFDE
:1007B00007F006503E24026E07503F20036E000EE5
:1007C0004020046E000E4120056E05C06CF004C090
:1007D0006BF003C06AF002C069F02A8E06D02C9E2E
:1007E0002A9E6C686B686A68696802D020685ED06F
:1007F00020685BD05BD059D0A20E1D5C0CE1222892
:1008000003E11BC022F005D01BC023F021EC06F051
:100810004CD04CD04AD0B20E1D5C1EE1242803E11E
:100820001BC024F017D01BC025F01E0E245C06E070
:10083000420E245C03E07B0E245C09E1B20EEDEC79
:1008400000F02450EDEC00F02550EDEC00F05CECF5
:1008500006F02BD02BD029D0C20E1D5C10E126282B
:100860000CE11BC026F0080E265C06E2C20EEDEC81
:1008700000F02650EDEC00F0266818D016D0D20E0D
:100880001D5C07E1272803E11BC027F027680ED075
:100890000CD0E20E1D5C09E1282803E11BC028F002
:1008A00003D01BC029F0286801D091D9080E485CFC
:1008B000D8B084D144503E5C45503F5846504058D3
:1008C00047504158D8A06CD1478E48522EE18078CD
:1008D000929880B815D03A503E24026E3B503F208B
:1008E000036E3C504020046E3D504120056E05C013
:1008F00050F004C04FF003C04EF002C04DF014D0D1
:1009000036503E24026E37503F20036E3850402050
:10091000046E39504120056E05C050F004C04FF000
:1009200003C04EF002C04DF03AD1010E485C2AE1FE
:100930002CB206D08B9A546853685268516821D003
:10094000827A949A02EE6DF0D8902F34E926000E48
:10095000EA22EECF06F0EFCF07F006503E24026EFB
:1009600007503F20036E000E4020046E000E412011
:10097000056E05C054F004C053F003C052F002C02D
:1009800051F00DD1020E485C2AE12CB406D0899AB0
:10099000586857685668556821D0807A929A02EE56
:1009A0006DF0D8903034E926000EEA22EECF06F042
:1009B000EFCF07F006503E24026E07503F20036E33
:1009C000000E4020046E000E4120056E05C058F058
:1009D00004C057F003C056F002C055F0E0D0030E3B
:1009E000485C2AE12CB606D08B905C685B685A683C
:1009F000596821D08270949002EE6DF0D890313415
:100A0000E926000EEA22EECF06F0EFCF07F00650FF
:100A10003E24026E07503F20036E000E4020046EFD
:100A2000000E4120056E05C05CF004C05BF003C001
:100A30005AF002C059F0B3D0040E485C2AE12CB839
:100A400006D08B9260685F685E685D6821D08272B4
:100A5000949202EE6DF0D8903234E926000EEA222C
:100A6000EECF06F0EFCF07F006503E24026E07509F
:100A70003F20036E000E4020046E000E4120056EE4
:100A800005C060F004C05FF003C05EF002C05DF01E
:100A900086D0050E485C2AE12CBA06D08B94646897
:100AA00063686268616821D08274949402EE6DF08C
:100AB000D8903334E926000EEA22EECF06F0EFCFCD
:100AC00007F006503E24026E07503F20036E000ED2
:100AD0004020046E000E4120056E05C064F004C085
:100AE00063F003C062F002C061F059D0060E485CAA
:100AF0002AE12CBC06D08B966868676866686568D2
:100B000021D08276949602EE6DF0D8903434E926A6
:100B1000000EEA22EECF06F0EFCF07F006503E249B
:100B2000026E07503F20036E000E4020046E000E40
:100B30004120056E05C068F004C067F003C066F090
:100B400002C065F02CD0070E485C29E12CBE06D00F
:100B50008B986C686B686A68696821D08278949811
:100B600002EE6DF0D8903534E926000EEA22EECF81
:100B700006F0EFCF07F006503E24026E07503F20EC
:100B8000036E000E4020046E000E4120056E05C06D
:100B90006CF004C06BF003C06AF002C069F017D8B3
:100BA00041AE0BD0416A406A3F6A3E6A2C6A00EE51
:100BB0004DF0200EEE68E82EFDD706D041AE04D0F1
:100BC000416A406A3F6A3E6A817030EF01F04868CE
:100BD000478E1C6A080E1C5C33E2D8901C34E96E08
:100BE000EA6AEA36E936EA364D0EE926000EEA22CE
:100BF000EFCF02F0ECCF03F0ECCF04F0ECCF05F038
:100C00004450025C4550035846500458475005581C
:100C100015E2D8901C34E96EEA6AEA36E936EA361B
:100C20004D0EE926000EEA22EFCF44F0ECCF45F05E
:100C3000ECCF46F0ECCF47F01CC048F01C2ACAE3CA
:100C40001200240E225C0DE3650E225C0AE2A20E65
:100C5000EDEC00F02250EDEC00F02350EDEC00F054
:100C600029D07C0E225C03E123C02FF023D07D0E1F
:100C7000225C03E123C030F01DD07E0E225C03E134
:100C800023C031F017D07F0E225C03E123C032F085
:100C900011D0750E225C03E123C033F00BD0760E29
:100CA000225C03E123C034F005D0770E225C02E120
:100CB00023C035F022681200070E245CD8A459D056
:100CC0002BA050D0D8902534E96EEA6AEA36E9368E
:100CD000EA366D0EE926060EEA22EFCF36F0ECCFAB
:100CE00037F0ECCF38F0ECCF39F0D8902534E96EFE
:100CF000EA6AEA36E936EA366D0EE926040EEA2299
:100D0000EFCF3AF0ECCF3BF0ECCF3CF0ECCF3DF046
:100D1000255207E1899850684F684E684D682A90BF
:100D200020D07D0E255C07E3898850684F684E68A7
:100D30004D682A9016D0898836503E24026E37506E
:100D40003F20036E38504020046E39504120056E1C
:100D500005C050F004C04FF003C04EF002C04DF08B
:100D60002A8006D0899850684F684E684D682A904E
:100D700032D01E0E245C11E12BA00ED025C02FF026
:100D800025C030F025C031F025C032F025C033F049
:100D900025C034F025C035F01ED0420E245C09E198
:100DA000255204E18A942B9018D802D08A842B8093
:100DB00012D07B0E245C0FE12C6A8B928B948B9665
:100DC0008B988B9A899A8B902A922A942A962A98A1
:100DD0002A9A2A9C2A9E24681200899850684F6893
:100DE0004E684D682A908A942A6A2C6A2F6A306A63
:100DF000316A326A336A346A356A8B928B948B9685
:100E00008B988B9A899A8B902B6A120002016E69DB
:100E10006D695C0E706F7A0E6F6F590E726F850E72
:100E2000716F580E746F140E736F560E766FA90E95
:100E3000756F550E786F430E776F530E7A6FE30E12
:100E4000796F520E7C6F890E7B6F510E7E6F350E5F
:100E50007D6F4F0E806FE60E7F6F4E0E826F9C0E81
:100E6000816F4D0E846F580E836F4C0E866F190E76
:100E7000856F4A0E886FDF0E876F490E8A6FAA0E44
:100E8000896F480E8C6F7A0E8B6F470E8E6F4F0EE8
:100E90008D6F460E906F290E8F6F450E926F080E64
:100EA000916F430E946FEB0E936F420E966FD30EBD
:100EB000956F410E986FBF0E976F400E9A6FB00EF0
:100EC000996F3F0E9C6FA50E9B6F3E0E9E6F9E0E00
:100ED0009D6F3D0EA06F9C0E9F6F3C0EA26F9E0EED
:100EE000A16F3B0EA46FA40EA36F3A0EA66FAE0EB9
:100EF000A56F390EA86FBC0EA76F380EAA6FCE0E65
:100F0000A96F370EAC6FE30EAB6F360EAE6FFD0EF2
:100F1000AD6F360EB06F1A0EAF6F350EB26F3B0E5F
:100F2000B16F340EB46F5F0EB36F330EB66F870EB2
:100F3000B56F320EB86FB20EB76F310EBA6FE10EE9
:100F4000B96F310EBC6F140EBB6F300EBE6F490E01
:100F5000BD6F2F0EC06F820EBF6F2E0EC26FBE0E02
:100F6000C16F2D0EC46FFD0EC36F2D0EC66F3F0EE9
:100F7000C56F2C0EC86F850EC76F2B0ECA6FCD0EB6
:100F8000C96F2B0ECC6F180ECB6F2A0ECE6F670E6B
:100F9000CD6F290ED06FB80ECF6F290ED26F0C0E09
:100FA000D16F280ED46F620ED36F270ED66FBC0E92
:100FB000D56F270ED86F180ED76F260EDA6F760E04
:100FC000D96F250EDC6FD80EDB6F250EDE6F3C0E61
:100FD000DD6F240EE06FA20EDF6F240EE26F0B0EAA
:100FE000E16F230EE46F760EE36F220EE66FE40EE0
:100FF000E56F220EE86F540EE76F210EEA6FC60E02
:10100000E96F210EEC6F3B0EEB6F200EEE6FB20E10
:10101000ED6F200EF06F2B0EEF6F1F0EF26FA60E0E
:10102000F16F1F0EF46F240EF36F1E0EF66FA30EFA
:10103000F56F1E0EF86F250EF76F1D0EFA6FA90ED5
:10104000F96F1D0EFC6F2E0EFB6F1C0EFE6FB60EA1
:10105000FD6F1C0E0301006F3F0E0201FF6F1B0EA0
:101060000301026FCB0E016F1B0E046F580E036F4E
:101070001A0E066FE80E056F1A0E086F790E076FCD
:101080001A0E0A6F0B0E096F190E0C6FA00E0B6F64
:10109000190E0E6F360E0D6F180E106FCE0E0F6FED
:1010A000180E126F680E116F180E146F030E136F67
:1010B000170E166FA00E156F170E186F3F0E176FD5
:1010C000160E1A6FDF0E196F160E1C6F800E1B6F37
:1010D000160E1E6F240E1D6F150E206FC80E1F6F8B
:1010E000150E226F6E0E216F150E246F160E236FD4
:1010F000140E266FBF0E256F140E286F690E276F12
:10110000140E2A6F150E296F130E2C6FC20E2B6F43
:10111000130E2E6F710E2D6F130E306F210E2F6F69
:10112000120E326FD20E316F120E346F840E336F87
:10113000120E366F380E356F110E386FED0E376F99
:10114000110E3A6FA30E396F110E3C6F5A0E3B6FA2
:10115000110E3E6F120E3D6F100E406FCC0E3F6FA2
:10116000100E426F870E416F100E446F420E436F98
:101170000F0E466F4569486FBD0E476F0F0E4A6FE1
:101180007C0E496F0F0E4C6F3D0E4B6F0E0E4E6F67
:10119000FE0E4D6F0E0E506FC00E4F6F0E0E526F43
:1011A000830E516F0E0E546F470E536F0E0E566F17
:1011B0000C0E556F0D0E586FD20E576F0D0E5A6FE5
:1011C000990E596F0D0E5C6F610E5B6F0D0E5E6FA9
:1011D0002A0E5D6F0C0E606FF40E5F6F0C0E626F67
:1011E000BE0E616F0C0E646F8A0E636F0C0E666F1D
:1011F000560E656F0C0E686F230E676F0B0E6A6FCD
:10120000F10E696F0B0E6C6FC00E6B6F6E696D69BE
:10121000A20E706FC30E6F6F9A0E726F460E716FD3
:10122000960E746F320E736F920E766F3A0E756F64
:101230008E0E786F5D0E776F8A0E7A6F9A0E796FC9
:10124000860E7C6FF00E7B6F830E7E6F5F0E7D6F60
:101250007F0E806FE70E7F6F7C0E826F850E816F31
:10126000790E846F3B0E836F760E866F070E856F47
:10127000720E886FE80E876F6F0E8A6FDF0E896FB0
:101280006C0E8C6FEA0E8B6F6A0E8E6F0A0E8D6F6E
:10129000670E906F3C0E8F6F640E926F820E916F8F
:1012A000610E946FDA0E936F5F0E966F440E956F1A
:1012B0005C0E986FBF0E976F5A0E9A6F4C0E996F17
:1012C000570E9C6FE90E9B6F550E9E6F960E9D6F8D
:1012D000530EA06F9F6F510EA26F200EA16F4E0E86
:1012E000A46FFB0EA36F4C0EA66FE50EA56F4A0E02
:1012F000A86FDC0EA76F480EAA6FE20EA96F460E0C
:10130000AC6FF50EAB6F450EAE6F150EAD6F430EA5
:10131000B06F420EAF6F410EB26F7B0EB16F3F0EDA
:10132000B46FC00EB36F3E0EB66F100EB56F3C0EAD
:10133000B86F6D0EB76F3A0EBA6FD40EB96F390E23
:10134000BC6F460EBB6F370EBE6FC20EBD6F360E42
:10135000C06F490EBF6F340EC26FDA0EC16F330E0D
:10136000C46F740EC36F320EC66F180EC56F300E89
:10137000C86FC50EC76F2F0ECA6F7B0EC96F2E0EBA
:10138000CC6F3A0ECB6F2D0ECE6F020ECD6F2B0EA3
:10139000D06FD10ECF6F2A0ED26FA90ED16F290E4A
:1013A000D46F880ED36F280ED66F6F0ED56F270EB1
:1013B000D86F5E0ED76F260EDA6F530ED96F250EDB
:1013C000DC6F500EDB6F240EDE6F540EDD6F230ECC
:1013D000E06F5E0EDF6F220EE26F6F0EE16F210E87
:1013E000E46F860EE36F200EE66FA30EE56F1F0E0F
:1013F000E86FC60EE76F1E0EEA6FEF0EE96F1E0E66
:10140000EC6FEB6F1D0EEE6F520EED6F1C0EF06F5A
:101410008C0EEF6F1B0EF26FCB0EF16F1B0EF46F85
:101420000F0EF36F1A0EF66F580EF56F190EF86F58
:10143000A50EF76F180EFA6FF80EF96F180EFC6F05
:101440004F0EFB6F170EFE6FAB0EFD6F170E0401F4
:10145000006F0A0E0301FF6F160E0401026F6F0E7C
:10146000016F150E046FD70E036F150E066F430E36
:10147000056F140E086FB30E076F140E0A6F270E58
:10148000096F130E0C6F9F0E0B6F130E0E6F1A0E5B
:101490000D6F120E106F990E0F6F120E126F1B0E42
:1014A000116F110E146FA10E136F110E166F290E0E
:1014B000156F100E186FB50E176F100E1A6F440EC1
:1014C000196F0F0E1C6FD60E1B6F0F0E1E6F6B0E5B
:1014D0001D6F0F0E206F030E1F6F0E0E226F9D0EDD
:1014E000216F0E0E246F3A0E236F0D0E266FDA0E4B
:1014F000256F0D0E286F7C0E276F0D0E2A6F210EA3
:10150000296F0C0E2C6FC80E2B6F0C0E2E6F720EE7
:101510002D6F0C0E306F1E0E2F6F0B0E326FCC0E18
:10152000316F0B0E346F7C0E336F0B0E366F2E0E39
:10153000356F0A0E386FE30E376F0A0E3A6F990E49
:10154000396F0A0E3C6F510E3B6F0A0E3E6F0B0E49
:101550003D6F090E406FC80E3F6F090E426F850E3A
:10156000416F090E446F450E436F090E466F060E1C
:10157000456F080E486FC90E476F080E4A6F8E0EF2
:10158000496F080E4C6F540E4B6F080E4E6F1C0EB9
:101590004D6F070E506FE50E4F6F070E526FAF0E77
:1015A000516F070E546F7B0E536F070E566F490E27
:1015B000556F070E586F170E576F060E5A6FE70ECE
:1015C000596F060E5C6FB90E5B6F060E5E6F8B0E69
:1015D0005D6F060E606F5F0E5F6F060E626F340EFA
:1015E000616F060E646F0A0E636F050E666FE10E83
:1015F000656F050E686FB90E676F050E6A6F930E03
:10160000696F050E6C6F6D0E6B6F00011200040E9A
:101610000101706F880E6F6F040E726FA60E716FEE
:10162000040E746FB60E736F040E766FC60E756F70
:10163000040E786FD60E776F040E7A6FE60E796F10
:10164000040E7C6FF60E7B6F050E7E6F070E7D6FAE
:10165000050E806F170E7F6F050E826F280E816F4B
:10166000050E846F390E836F050E866F4B0E856FE6
:10167000050E886F5D0E876F050E8A6F6E0E896F7F
:10168000050E8C6F800E8B6F050E8E6F930E8D6F17
:10169000050E906FA50E8F6F050E926FB80E916FAD
:1016A000050E946FCB0E936F050E966FDF0E956F40
:1016B000050E986FF20E976F060E9A6F996F9C6FDA
:1016C0001A0E9B6F060E9E6F2E0E9D6F060EA06F5C
:1016D000430E9F6F060EA26F580EA16F060EA46FE9
:1016E0006D0EA36F060EA66F830EA56F060EA86F74
:1016F000980EA76F060EAA6FAE0EA96F060EAC6FFE
:10170000C40EAB6F060EAE6FDB0EAD6F060EB06F84
:10171000F20EAF6F070EB26F090EB16F070EB46F06
:10172000210EB36F070EB66F380EB56F070EB86F88
:10173000500EB76F070EBA6F690EB96F070EBC6F08
:10174000810EBB6F070EBE6F9A0EBD6F070EC06F86
:10175000B40EBF6F070EC26FCD0EC16F070EC46F00
:10176000E70EC36F080EC66F020EC56F080EC86F76
:101770001D0EC76F080ECA6F380EC96F080ECC6FEA
:10178000530ECB6F080ECE6F6F0ECD6F080ED06F5D
:101790008B0ECF6F080ED26FA70ED16F080ED46FCD
:1017A000C40ED36F080ED66FE10ED56F080ED86F3A
:1017B000D769090EDA6F1D0ED96F090EDC6F3B0E6B
:1017C000DB6F090EDE6F5A0EDD6F090EE06F790ECA
:1017D000DF6F090EE26F990EE16F090EE46FB90E2B
:1017E000E36F090EE66FD90EE56F090EE86FFA0E8A
:1017F000E76F0A0EEA6F1B0EE96F0A0EEC6F3D0EE3
:10180000EB6F0A0EEE6F5F0EED6F0A0EF06F820E39
:10181000EF6F0A0EF26FA50EF16F0A0EF46FC80E8D
:10182000F36F0A0EF66FEC0EF56F0B0EF86F110EDC
:10183000F76F0B0EFA6F360EF96F0B0EFC6F5B0E27
:10184000FB6F0B0EFE6F810EFD6F0B0E0201006F22
:10185000A70E0101FF6F0B0E0201026FCE0E016F8A
:101860000B0E046FF50E036F0C0E066F1D0E056F49
:101870000C0E086F460E076F0C0E0A6F6F0E096F85
:101880000C0E0C6F980E0B6F0C0E0E6FC20E0D6FC0
:101890000C0E106FED0E0F6F0D0E126F180E116FF4
:1018A0000D0E146F430E136F0D0E166F700E156F25
:1018B0000D0E186F9C0E176F0D0E1A6FCA0E196F52
:1018C0000D0E1C6FF80E1B6F0E0E1E6F260E1D6F79
:1018D0000E0E206F550E1F6F0E0E226F850E216F9C
:1018E0000E0E246FB60E236F0E0E266FE70E256FB9
:1018F0000F0E286F180E276F0F0E2A6F4B0E296FD1
:101900000F0E2C6F7E0E2B6F0F0E2E6FB10E2D6FE4
:101910000F0E306FE60E2F6F100E326F1B0E316FF1
:10192000100E346F500E336F100E366F870E356FFA
:10193000100E386FBE0E376F100E3A6FF60E396FFD
:10194000110E3C6F2E0E3B6F110E3E6F680E3D6FF9
:10195000110E406FA20E3F6F110E426FDC0E416FF1
:10196000120E446F180E436F120E466F540E456FE1
:10197000120E486F910E476F120E4A6FCF0E496FCD
:10198000130E4C6F0E0E4B6F130E4E6F4D0E4D6FB0
:10199000130E506F8E0E4F6F130E526FCF0E516F8E
:1019A000140E546F110E536F140E566F540E556F64
:1019B000140E586F980E576F140E5A6FDC0E596F35
:1019C000150E5C6F220E5B6F150E5E6F680E5D6FFD
:1019D000150E606FB00E5F6F150E626FF80E616FBF
:1019E000160E646F410E636F160E666F8C0E656F78
:1019F000160E686FD70E676F170E6A6F230E696F2A
:101A0000170E6C6F700E6B6F000112000601746B85
:101A1000736B726B020E716F0401746B736B726B7C
:101A2000300E716F0601786B776B766B020E756FF7
:101A30000401786B776B766B300E756F06017C6BEB
:101A40007B6B7A6B020E796F04017C6B7B6B7A6B1C
:101A5000300E796F0601806B7F6B7E6B020E7D6F9F
:101A60000401806B7F6B7E6B170E7D6F0601846BAC
:101A7000836B826B020E816F0401846B836B826BBC
:101A8000170E816F0601886B876B866B020E856F60
:101A90000401886B876B866B170E856F06018C6B54
:101AA0008B6B8A6B020E896F04018C6B8B6B8A6B5C
:101AB000170E896F0601906B8F6B8E6B020E8D6F08
:101AC0000401906B8F6B8E6B170E8D6F0601946BFC
:101AD000936B926B020E916F0401946B936B926BFC
:101AE000170E916F0601986B976B966B060E956FAC
:101AF0000401986B976B966B2C0E956F06019C6B8F
:101B00009B6B9A6B060E996F04019C6B9B6B9A6B97
:101B10002C0E996F0601A06B9F6B9E6B060E9D6F3E
:101B20000401A06B9F6B9E6B2C0E9D6F0601A46B36
:101B3000A36BA26B060EA16F0401A46BA36BA26B37
:101B40002C0EA16F0601A86BA76BA66B060EA56FE6
:101B50000401A86BA76BA66B2C0EA56F0601AC6BDE
:101B6000AB6BAA6B040EA96F0401AC6BAB6BAA6BD9
:101B7000150EA96F0601B06BAF6BAE6B040EAD6FA7
:101B80000401B06BAF6BAE6B150EAD6F0601B46B9D
:101B9000B36BB26B040EB16F0401B46BB36BB26B79
:101BA000150EB16F0601B86BB76BB66B040EB56F4F
:101BB0000401B86BB76BB66B150EB56F0601BC6B45
:101BC000BB6BBA6B040EB96F0401BC6BBB6BBA6B19
:101BD000150EB96F0601C06BBF6BBE6B0A0EBD6FF1
:101BE0000401C06BBF6BBE6B280EBD6F0601C46BDA
:101BF000C36BC26B0A0EC16F0401C46BC36BC26BB3
:101C0000280EC16F0601C86BC76BC66B0A0EC56F85
:101C10000401C86BC76BC66B280EC56F0601CC6B81
:101C2000CB6BCA6B0A0EC96F0401CC6BCB6BCA6B52
:101C3000280EC96F0601D06BCF6BCE6B0A0ECD6F2D
:101C40000401D06BCF6BCE6B280ECD6F0601D46B29
:101C5000D36BD26B060ED16F0401D46BD36BD26BF6
:101C6000130ED16F0601D86BD76BD66B060ED56FEE
:101C70000401D86BD76BD66B130ED56F0601DC6BE6
:101C8000DB6BDA6B060ED96F0401DC6BDB6BDA6B96
:101C9000130ED96F0601E06BDF6BDE6B060EDD6F96
:101CA0000401E06BDF6BDE6B130EDD6F0601E46B8E
:101CB000E36BE26B060EE16F0401E46BE36BE26B36
:101CC000130EE16F0601E86BE76BE66B060EE56F3E
:101CD0000401E86BE76BE66B130EE56F0601EC6B36
:101CE000EB6BEA6B0E0EE96F0401EC6BEB6BEA6BCE
:101CF000240EE96F0601F06BEF6BEE6B0E0EED6FCD
:101D00000401F06BEF6BEE6B240EED6F0601F46BCC
:101D1000F36BF26B0E0EF16F0401F46BF36BF26B6D
:101D2000240EF16F0601F86BF76BF66B0E0EF56F74
:101D30000401F86BF76BF66B240EF56F0601FC6B74
:101D4000FB6BFA6B0E0EF96F0401FC6BFB6BFA6B0D
:101D5000240EF96F0701006B0601FF6BFE6B080E86
:101D6000FD6F0501006B0401FF6BFE6B110EFD6F33
:101D70000701046B036B026B080E016F0501046B16
:101D8000036B026B110E016F0701086B076B066B8B
:101D9000080E056F0501086B076B066B110E056FCA
:101DA00007010C6B0B6B0A6B080E096F05010C6BBE
:101DB0000B6B0A6B110E096F0701106B0F6B0E6B2B
:101DC000080E0D6F0501106B0F6B0E6B110E0D6F72
:101DD0000701146B136B126B120E116F0501146B5C
:101DE000136B126B200E116F0701186B176B166BBC
:101DF000120E156F0501186B176B166B200E156F01
:101E000007011C6B1B6B1A6B120E196F05011C6B03
:101E10001B6B1A6B200E196F0701206B1F6B1E6B5B
:101E2000120E1D6F0501206B1F6B1E6B200E1D6FA8
:101E30000701246B236B226B120E216F0501246BAB
:101E4000236B226B200E216F0701286B276B266BFB
:101E50000A0E256F0501286B276B266B0F0E256F69
:101E600007012C6B2B6B2A6B0A0E296F05012C6B5B
:101E70002B6B2A6B0F0E296F0701306B2F6B2E6BAC
:101E80000A0E2D6F0501306B2F6B2E6B0F0E2D6F11
:101E90000701346B336B326B0A0E316F0501346B03
:101EA000336B326B0F0E316F0701386B376B366B4C
:101EB0000A0E356F0501386B376B366B0F0E356FB9
:101EC00007013C6B3B6B3A6B0A0E396F05013C6BAB
:101ED0003B6B3A6B0F0E396F0701406B3F6B3E6BEC
:101EE000160E3D6F0501406B3F6B3E6B1C0E3D6F48
:101EF0000701446B436B426B160E416F0501446B47
:101F0000436B426B1C0E416F0701486B476B466B7E
:101F1000160E456F0501486B476B466B1C0E456FEF
:101F200007014C6B4B6B4A6B160E496F05014C6BEE
:101F30004B6B4A6B1C0E496F0701506B4F6B4E6B1E
:101F4000160E4D6F0501506B4F6B4E6B1C0E4D6F97
:101F50000701546B536B526B0C0E516F0501546BA0
:101F6000536B526B0D0E516F0701586B576B566BCD
:101F70000C0E556F0501586B576B566B0D0E556F58
:101F800007015C6B5B6B5A6B0C0E596F05015C6B48
:101F90005B6B5A6B0D0E596F0701606B5F6B5E6B6D
:101FA0000C0E5D6F0501606B5F6B5E6B0D0E5D6F00
:101FB0000701646B636B626B0C0E616F0501646BF0
:101FC000636B626B0D0E616F0701686B676B666B0D
:101FD0001A0E656F0501686B676B666B180E656F8F
:101FE00007016C6B6B6B6A6B1A0E696F05016C6B8A
:101FF0006B6B6A6B180E696F0701706B6F6B6E6BA2
:102000001A0E6D6F0501706B6F6B6E6B180E6D6F36
:102010000701746B736B726B1A0E716F0501746B31
:10202000736B726B180E716F0701786B776B766B41
:102030001A0E756F0501786B776B766B180E756FDE
:1020400007017C6B7B6B7A6B0E0E796F05017C6BE5
:102050007B6B7A6B0B0E796F0701806B7F6B7E6BEE
:102060000E0E7D6F0501806B7F6B7E6B0B0E7D6F9F
:102070000701846B836B826B0E0E816F0501846B8D
:10208000836B826B0B0E816F0701886B876B866B8E
:102090000E0E856F0501886B876B866B0B0E856F47
:1020A00007018C6B8B6B8A6B0E0E896F05018C6B35
:1020B0008B6B8A6B0B0E896F0701906B8F6B8E6B2E
:1020C0000E0E8D6F0501906B8F6B8E6B0B0E8D6FEF
:1020D0000701946B936B926B1E0E916F0501946BCD
:1020E000936B926B140E916F0701986B976B966BC5
:1020F0001E0E956F0501986B976B966B140E956F7E
:1021000007019C6B9B6B9A6B1E0E996F05019C6B74
:102110009B6B9A6B140E996F0701A06B9F6B9E6B64
:102120001E0E9D6F0501A06B9F6B9E6B140E9D6F25
:102130000701A46BA36BA26B1E0EA16F0501A46B1C
:10214000A36BA26B140EA16F0701A86BA76BA66B04
:10215000100EA56F0501A86BA76BA66B090EA56FE6
:102160000701AC6BAB6BAA6B100EA96F0501AC6BD2
:10217000AB6BAA6B090EA96F0701B06BAF6BAE6BAF
:10218000100EAD6F0501B06BAF6BAE6B090EAD6F8E
:102190000701B46BB36BB26B100EB16F0501B46B7A
:1021A000B36BB26B090EB16F0701B86BB76BB66B4F
:1021B000100EB56F0501B86BB76BB66B090EB56F36
:1021C0000701BC6BBB6BBA6B220EB96F0501BC6B10
:1021D000BB6BBA6B100EB96F0701C06BBF6BBE6BE8
:1021E000220EBD6F0501C06BBF6BBE6B100EBD6FC5
:1021F0000701C46BC36BC26B220EC16F0501C46BB8
:10220000C36BC26B100EC16F0701C86BC76BC66B87
:10221000220EC56F0501C86BC76BC66B100EC56F6C
:102220000701CC6BCB6BCA6B220EC96F0501CC6B5F
:10223000CB6BCA6B100EC96F0701D06BCF6BCE6B27
:10224000120ECD6F0501D06BCF6BCE6B070ECD6F2D
:102250000701D46BD36BD26B120ED16F0501D46B17
:10226000D36BD26B070ED16F0701D86BD76BD66BD0
:10227000120ED56F0501D86BD76BD66B070ED56FD5
:102280000701DC6BDB6BDA6B120ED96F0501DC6BBF
:10229000DB6BDA6B070ED96F0701E06BDF6BDE6B70
:1022A000120EDD6F0501E06BDF6BDE6B070EDD6F7D
:1022B0000701E46BE36BE26B120EE16F0501E46B67
:1022C000E36BE26B070EE16F0701E86BE76BE66B10
:1022D000260EE56F0501E86BE76BE66B0C0EE56F0C
:1022E0000701EC6BEB6BEA6B260EE96F0501EC6BFB
:1022F000EB6BEA6B0C0EE96F0701F06BEF6BEE6BAB
:10230000260EED6F0501F06BEF6BEE6B0C0EED6FB3
:102310000701F46BF36BF26B260EF16F0501F46BA2
:10232000F36BF26B0C0EF16F0701F86BF76BF66B4A
:10233000260EF56F0501F86BF76BF66B0C0EF56F5B
:102340000701FC6BFB6BFA6B140EF96F0501FC6B5C
:10235000FB6BFA6B050EF96F0801006B0701FF6B51
:10236000FE6B140EFD6F0601006B0501FF6BFE6B2B
:10237000050EFD6F0801046B036B026B140E016FF9
:102380000601046B036B026B050E016F0801086BFD
:10239000076B066B140E056F0601086B076B066B67
:1023A000050E056F08010C6B0B6B0A6B140E096FA1
:1023B00006010C6B0B6B0A6B050E096F0801106BA5
:1023C0000F6B0E6B2A0E0D6F0601106B0F6B0E6BF1
:1023D000080E0D6F0801146B136B126B2A0E116F30
:1023E0000601146B136B126B080E116F0801186B4A
:1023F000176B166B2A0E156F0601186B176B166B91
:10240000080E156F08011C6B1B6B1A6B2A0E196FD7
:1024100006011C6B1B6B1A6B080E196F0801206BF1
:102420001F6B1E6B2A0E1D6F0601206B1F6B1E6B30
:10243000080E1D6F0801246B236B226B160E216F93
:102440000601246B236B226B030E216F0801286B9E
:10245000276B266B160E256F0601286B276B266BE4
:10246000030E256F08012C6B2B6B2A6B160E296F40
:1024700006012C6B2B6B2A6B030E296F0801306B46
:102480002F6B2E6B160E2D6F0601306B2F6B2E6B84
:10249000030E2D6F0801346B336B326B160E316FE8
:1024A0000601346B336B326B030E316F0801386BEE
:1024B000376B366B160E356F0601386B376B366B24
:1024C000030E356F08013C6B3B6B3A6B2E0E396F78
:1024D00006013C6B3B6B3A6B040E396F0801406B95
:1024E0003F6B3E6B2E0E3D6F0601406B3F6B3E6BAC
:1024F000040E3D6F0801446B436B426B2E0E416F1F
:102500000601446B436B426B040E416F0801486B3C
:10251000476B466B2E0E456F0601486B476B466B4B
:10252000040E456F08014C6B4B6B4A6B2E0E496FC6
:1025300006014C6B4B6B4A6B040E496F0801506BE4
:102540004F6B4E6B180E4D6F0601506B4F6B4E6B01
:10255000010E4D6F0801546B536B526B180E516F87
:102560000601546B536B526B010E516F0801586B8F
:10257000576B566B180E556F0601586B576B566BA1
:10258000010E556F08015C6B5B6B5A6B180E596F2F
:1025900006015C6B5B6B5A6B010E596F0801606B37
:1025A0005F6B5E6B180E5D6F0601606B5F6B5E6B41
:1025B000010E5D6F0801646B636B626B320E616FBD
:1025C0000601646B636B626B616B0801686B676B20
:1025D000666B656F0601686B676B666B656B010EFA
:1025E0001C6E00017F0E1C5CD8B07DD0D8901C34CE
:1025F000E96EEA6AEA36E936EA366D0EE926060E33
:10260000EA22EFCF06F0ECCF07F0ECCF08F0ECCFEA
:1026100009F009C00DF008C00CF007C00BF006C0AF
:102620000AF0136A126A030E116EE80E106E25ECA2
:1026300000F00DC005F00CC004F00BC003F00AC0A0
:1026400002F01C50040DF3CFE9FFF4CFEAFF6D0E4A
:10265000E926060EEA2202C0EEFF03C0EEFF04C028
:10266000EEFF05C0EFFFD8901C34E96EEA6AEA3647
:10267000E936EA366D0EE926040EEA22EFCF06F0BF
:10268000ECCF07F0ECCF08F0ECCF09F009C00DF06B
:1026900008C00CF007C00BF006C00AF0136A126AFB
:1026A000030E116EE80E106E25EC00F00DC005F063
:1026B0000CC004F00BC003F00AC002F01C50040D63
:1026C000F3CFE9FFF4CFEAFF6D0EE926040EEA220C
:1026D00002C0EEFF03C0EEFF04C0EEFF05C0EFFF37
:0A26E0001C2AD8A07ED71200FFD7F5
:020000040030CA
:0300010006160ED2
:020005008580F4
:060008000FC00FE00F40E5
:00000001FF
